:020000040000FA
:0600000048EF14F01200AD
:020006001200E6
:060008000BEF0FF01200E7
:02000E00C2909E
:040010009D9C1200A1
:04001400B46A1200B8
:060018006FEF0FF0120073
:02001E000200DE
:10002000F3280000DF07000011000000E2280000B4
:08003000DF06000011000000D2
:08003800D9CFE6FFE1CFD9FFAB
:10004000FD0EDBCFFCF6FE0EDBCFFDF6FCC6E9FFB6
:10005000FDC6EAFFDC0EE926000EEA22EE6AED6A32
:10006000FCC6E9FFFDC6EAFFE00EE926000EEA2223
:10007000EF6AFCC6E9FFFDC6EAFFDE0EE926000EC8
:10008000EA22050EEF6EFCC6E9FFFDC6EAFFE20EAE
:10009000E926000EEA22EF6AFCC6E9FFFDC6EAFF88
:1000A000DF0EE926000EEA22EF6AFCC6E9FFFDC674
:1000B000EAFFDC0EE926000EEA22EE6AED6AFCC6D3
:1000C000E9FFFDC6EAFFE30EE926000EEA22EF6A29
:1000D000FCC6E9FFFDC6EAFFE50EE926000EEA22AE
:1000E000EF6AFCC6E9FFFDC6EAFFE60EE926000E50
:1000F000EA22EF6AFCC6E9FFFDC6EAFFE90EE9263F
:10010000000EEA22EF6AFCC6E9FFFDC6EAFFE70E31
:10011000E926000EEA22EF6AFCC6E9FFFDC6EAFF07
:10012000E80EE926000EEA22220EEF6EE552E7CF36
:10013000D9FF1200FCC6E9FFFDC6EAFFE90EE92679
:10014000000EEA22110EEF6E94869488C76AC66A82
:10015000C56AF00EC6140809C66E770EC86EC78E43
:10016000C68A1200D9CFE6FFE1CFD9FF020EE12601
:10017000FD0EDB5069E0DE6ADD6ADECF10F0DDCF18
:1001800011F0FD0EDB50000111AE02D0D89003D06B
:10019000105C000E115820E2FB0EDBCF12F0FC0EBB
:1001A000DBCF13F0DE501224E96EDD501320EA6E2F
:1001B000EF50E66EFCC610F0FDC611F0DE501024C4
:1001C000E96EDD501120EA6EE552E750EF6EDF2A4E
:1001D000010ED3E3DB2AD1D7FD0EDB50E66EFCC661
:1001E000E9FFFDC6EAFFDC0EE926000EEA22E55231
:1001F000E750EE6EED6AFCC6E9FFFDC6EAFFE70ECA
:10020000E926000EEA22FE0EDBCFEFFFFCC6E9FF77
:10021000FDC6EAFFDF0EE926000EEA22EF6AFCC601
:10022000E9FFFDC6EAFFDE0EE926000EEA22090E0E
:10023000EF6EFCC6E9FFFDC6EAFFE80EE926000EF8
:10024000EA22200EEF6EC580020EE15C02E2E16A56
:10025000E552E16EE552E7CFD9FF1200D9CFE6FFB4
:10026000E1CFD9FFFD0EDB5038E0FD0EDB50E66E2E
:10027000FCC6E9FFFDC6EAFFDC0EE926000EEA2215
:10028000E552E750EE6EED6AFCC6E9FFFDC6EAFFF7
:10029000E70EE926000EEA22FE0EDBCFEFFFFCC6DA
:1002A000E9FFFDC6EAFFDF0EE926000EEA22EF6A4B
:1002B000FCC6E9FFFDC6EAFFDE0EE926000EEA22D3
:1002C000090EEF6EFCC6E9FFFDC6EAFFE80EE9265F
:1002D000000EEA22210EEF6EC580E552E7CFD9FF6E
:1002E0001200D9CFE6FFE1CFD9FFFCC6E9FFFDC67A
:1002F000EAFFE90EE926000EEA22100EEF6E948660
:100300009488FE0EDB50E824C86EC76AC66AC56AC8
:10031000F00EC6140E09C66EC78EC580C68AE55299
:10032000E7CFD9FF1200FCC6E9FFFDC6EAFFE90EE0
:10033000E926000EEA22EF50110802E1ADEF01F0CC
:10034000FCC6E9FFFDC6EAFFE90EE926000EEA2237
:10035000EF50100801E10CDA1200FCC6E9FFFDC6FF
:10036000EAFFE80EE926000EEA22EF50200801E03D
:10037000ADD0FCC6E9FFFDC6EAFFDE0EE926000EA1
:10038000EA22EF500B0A1CE0020A04E00C0A01E129
:100390009CD01200FCC6E9FFFDC6EAFFDE0EE9268E
:1003A000000EEA220B0EEF6EFCC6E9FFFDC6EAFF67
:1003B000E70EE926000EEA22EF50E824C96E12008B
:1003C000C5BC62D0FCC6E9FFFDC6EAFFDF0EE92628
:1003D000000EEA22EF50106E116AFCC6E9FFFDC65E
:1003E000EAFFDC0EE926000EEA22EECF12F0EFCF94
:1003F00013F011501318E8AE02D0133404D0125089
:10040000105C135011581EE2FCC6E9FFFDC6EAFF5E
:10041000FCC610F0FDC611F0DF0EE926000EEA2240
:10042000EF501024E96E000E1120EA6EEF50C96EF5
:10043000FCC6E9FFFDC6EAFFDF0EE926000EEA2250
:10044000EF2A1200FCC6E9FFFDC6EAFFDE0EE92630
:10045000000EEA22050EEF6EC584FCC6E9FFFDC65C
:10046000EAFFE80EE926000EEA22220EEF6E000EE9
:10047000E66EE66A2B0EE66EE66A80EC09F0E5525F
:10048000E552E552E5521200FCC6E9FFFDC6EAFF5F
:10049000DE0EE926000EEA22050EEF6EC584FCC6CC
:1004A000E9FFFDC6EAFFE80EE926000EEA22220E69
:1004B000EF6E000EE66EE66A2C0EE66EE66A80ECE3
:1004C00009F0E552E552E552E5521200FCC6E9FF9B
:1004D000FDC6EAFFE80EE926000EEA22EF502108E9
:1004E00001E0E7D0FCC6E9FFFDC6EAFFDE0EE92623
:1004F000000EEA22EF500D0A01E1ACD0010A01E141
:100500009DD00B0A43E00C0A1DE0020A04E00C0A2D
:1005100001E1CFD01200FCC6E9FFFDC6EAFFDE0E06
:10052000E926000EEA220B0EEF6EFCC6E9FFFDC6BF
:10053000EAFFE70EE926000EEA22EF50E82401095F
:10054000C96E1200C5AC7AD0FCC6E9FFFDC6EAFF51
:10055000DE0EE926000EEA22050EEF6EC584FCC60B
:10056000E9FFFDC6EAFFE80EE926000EEA22220EA8
:10057000EF6E000EE66EE66A2E0EE66EE66A80EC20
:1005800009F0E552E552E552E5521200FCC6E9FFDA
:10059000FDC6EAFFFCC610F0FDC611F0DF0EE9262D
:1005A000000EEA22EF501024E96E000E1120EA6ED0
:1005B000C9CFEFFFFCC6E9FFFDC6EAFFDF0EE92663
:1005C000000EEA22EF2AFCC6E9FFFDC6EAFFDF0EB5
:1005D000E926000EEA22EF50106E116AFCC6E9FF10
:1005E000FDC6EAFFDC0EE926000EEA22EECF12F08D
:1005F000EFCF13F011501318E8AE02D0133404D02B
:100600001250105C135011580CE2FCC6E9FFFDC6F5
:10061000EAFFDE0EE926000EEA220C0EEF6EC59A06
:100620000BD0FCC6E9FFFDC6EAFFDE0EE926000E90
:10063000EA220D0EEF6EC58AC5881200FCC6E9FFDE
:10064000FDC6EAFFDE0EE926000EEA22070EEF6E77
:10065000C5861200FCC6E9FFFDC6EAFFDE0EE926EC
:10066000000EEA22050EEF6EC584FCC6E9FFFDC64A
:10067000EAFFE80EE926000EEA22220EEF6EFCC623
:10068000E9FFFDC6EAFFFCC610F0FDC611F0FCC68E
:10069000E6FFFDC6E6FF2D0EE66EDC0EE926000E37
:1006A000EA22EF50E66E80EC09F0E552E552E552A1
:1006B000E5521200D9CFE6FFE1CFD9FFFCC6E9FF32
:1006C000FDC6EAFFE00EE926000EEA22010EEF6EFB
:1006D000FCC6E9FFFDC6EAFFDC0EE926000EEA22B1
:1006E000EE6AED6AFE0EDB5035E0C7AA1DD0FCC6EF
:1006F000E9FFFDC6EAFFDE0EE926000EEA22050E3E
:10070000EF6EFCC6E9FFFDC6EAFFE20EE926000E29
:10071000EA22EF2AFCC6E9FFFDC6EAFFE10EE92660
:10072000000EEA22050E1FD0C7A40AD0FCC6E9FFBE
:10073000FDC6EAFFDE0EE926000EEA22080E13D0FF
:10074000FCC6E9FFFDC6EAFFDE0EE926000EEA223E
:10075000070E09D0FCC6E9FFFDC6EAFFDE0EE9265A
:10076000000EEA22060EEF6EE552E7CFD9FF120027
:10077000D9CFE6FFE1CFD9FF090EE126010EDB6AF2
:10078000020EDB6A030EDB6A040EDB6A080EDB6A0C
:10079000C6AC23D0C69CFCC6E9FFFDC6EAFFDE0E50
:1007A000E926000EEA22050EEF6E010EF36E040E2E
:1007B000F3CFDBFFFCC6E9FFFDC6EAFFE20EE92648
:1007C000000EEA22EF2AFCC6E9FFFDC6EAFFE10EB1
:1007D000E926000EEA22040EEF6EC7A005D0C9502C
:1007E000DF6EDE52010EDD6E040EDB5001E03AD208
:1007F000FCC6E9FFFDC6EAFFDE0EE926000EEA228E
:10080000EF50070A01E17BD10F0A01E16FD00E0A18
:1008100017E0030A01E026D2C7A624D2010EDBCFDF
:10082000E6FF48DFE552FCC6E9FFFDC6EAFFDE0E43
:10083000E926000EEA22EF50080801E013D237D073
:10084000C7A810D0FCC6E9FFFDC6EAFFE00EE92606
:10085000000EEA22EF2A010EDB5001E1F9D1C7AA0E
:100860009CD1E3D1010EDB5001E1FCD1FCC6E9FFD4
:10087000FDC6EAFFE00EE926000EEA22EF2AC7BA1B
:1008800018D0C7B40AD0FCC6E9FFFDC6EAFFDE0EE9
:10089000E926000EEA22070EE4D1FCC6E9FFFDC6F8
:1008A000EAFFDE0EE926000EEA22080EEF6E030EC6
:1008B000BAD1FCC6E9FFFDC6EAFFE20EE926000E4A
:1008C000EA22EF2AFCC6E9FFFDC6EAFFDE0EE926B2
:1008D000000EEA22050EEF6EFCC6E9FFFDC6EAFF38
:1008E000E10EE926000EEA22060EBBD1FCC6E9FFA6
:1008F000FDC6EAFFE50EE926000EEA22EF5001E010
:100900007ED002EC0AF0E76E080EE7CFDBFFDB508B
:100910002A0803E1080EDB501BE1C968FCC6E9FFA9
:10092000FDC6EAFFDF0EE926000EEA22010EEF6E99
:10093000FCC6E9FFFDC6EAFFE50EE926000EEA2245
:10094000010EEF6EFCC6E9FFFDC6EAFFE60E51D0D0
:10095000FCC6E9FFFDC6EAFFFCC612F0FDC613F0B7
:10096000FCC6E6FFFDC6E6FFE40EE926000EEA221D
:10097000EF50E66EE66ADC0EE66EE2EC09F0146E0D
:10098000050EE15E1450106E116A10BE1168FCC6AF
:10099000E9FFFDC6EAFFDC0EE926000EEA2210C0E0
:1009A000EEFF11C0EDFFFCC6E9FFFDC6EAFFDC0E5D
:1009B000E926000EEA22EECF10F0EFCF11F011344D
:1009C00001E350D110500008000E115401E34AD148
:1009D000FCC6E9FFFDC6EAFFEF50C96EDF0EE9264F
:1009E000000EEA22010EEF6EFCC6E9FFFDC6EAFF2B
:1009F000E50EE926000EEA22010EEF6E71D0FCC66C
:100A0000E9FFFDC6EAFFE60EE926000EEA22EF50F6
:100A100026E0FCC6E9FFFDC6EAFFDF0EE926000E70
:100A2000EA22EFCF10F0FCC6E9FFFDC6EAFFE30EB5
:100A3000E926000EEA22EF50105C02E2C96846D0B7
:100A4000FCC6E9FFFDC6EAFFE50EE926000EEA2234
:100A5000EF6AFCC6E9FFFDC6EAFFE60E4BD0FCC616
:100A6000E9FFFDC6EAFFDF0EE926000EEA22EF509D
:100A7000106E116AFCC6E9FFFDC6EAFFDC0EE9262E
:100A8000000EEA22EECF12F0EFCF13F01150131840
:100A9000E8AE02D0133404D01250105C1350115839
:100AA00024E2FCC6E9FFFDC6EAFFFCC610F0FDC665
:100AB00011F0DF0EE926000EEA22EF500F0110249C
:100AC000E96E000E1120EA6EEF50C96EFCC6E9FF18
:100AD000FDC6EAFFDF0EE926000EEA22EF2A010E2C
:100AE000F36E020EF3CFDBFFBDD0FCC6E9FFFDC6FF
:100AF000EAFFE50EE926000EEA22EF6AA9D0C7A8B0
:100B000052D0FCC6E9FFFDC6EAFFE00EE926000E62
:100B1000EA22EF2A010EDB5040E0C7AA21D0FCC632
:100B2000E9FFFDC6EAFFFCC610F0FDC611F0DC0EC1
:100B3000E926000EEA221050EE24E76E1150EE2056
:100B4000EA6EE7CFE9FFDFCFEFFFFCC6E9FFFDC6A6
:100B5000EAFFDC0EE926000EEA22EE2AEF221DD083
:100B6000FCC6E9FFFDC6EAFFE20EE926000EEA2216
:100B7000EF2AFCC6E9FFFDC6EAFFE10EE926000EFA
:100B8000EA22060EEF6EFCC6E9FFFDC6EAFFDE0EA6
:100B9000E926000EEA22050E5AD0010EF36E030E6E
:100BA000F3CFDBFF55D0010EDB505CE0FCC6E9FF64
:100BB000FDC6EAFFE00EE926000EEA22EF2AC7AAE8
:100BC00021D0FCC6E9FFFDC6EAFFFCC610F0FDC659
:100BD00011F0DC0EE926000EEA221050EE24E76E3A
:100BE0001150EE20EA6EE7CFE9FFDFCFEFFFFCC642
:100BF000E9FFFDC6EAFFDC0EE926000EEA22EE2A36
:100C0000EF2230D0C7A411D0FCC6E9FFFDC6EAFF31
:100C1000DE0EE926000EEA22080EEF6E010EF36EDC
:100C2000030EF3CFDBFFC96E1DD0FCC6E9FFFDC686
:100C3000EAFFE20EE926000EEA22EF2AFCC6E9FFEF
:100C4000FDC6EAFFE10EE926000EEA22060EEF6E6F
:100C5000FCC6E9FFFDC6EAFFDE0EE926000EEA2229
:100C6000050EEF6E010EDB5003E1020EDB5002E0D9
:100C7000C6A8C688FCC6E9FFFDC6EAFFDC0EE92669
:100C8000000EEA22EECF10F0EFCF11F0113425E282
:100C90001050DA08000E115420E2030EDB501DE163
:100CA000FCC6E9FFFDC6EAFFDE0EE926000EEA22D9
:100CB000050EEF6EFCC6E9FFFDC6EAFFE20EE9266F
:100CC000000EEA22EF2AFCC6E9FFFDC6EAFFE10EAC
:100CD000E926000EEA22070EEF6E030EDB5070E0ED
:100CE000FCC6E9FFFDC6EAFFFCC610F0FDC611F028
:100CF000DC0EE926000EEA22EECF12F0EFCF13F061
:100D00001206135A10501224E96E11501320EA6E85
:100D1000EF50E66EFCC6E9FFFDC6EAFFE30EE926EA
:100D2000000EEA22E552E750EF6EFCC6E9FFFDC671
:100D3000EAFFE00EE926000EEA22EF50E66EFCC65E
:100D4000E9FFFDC6EAFFFCC610F0FDC611F0DC0E9F
:100D5000E926000EEA221050EE24E76E1150EE2034
:100D6000EA6EE7CFE9FFE552E750EF6EFCC6E9FF18
:100D7000FDC6EAFFFCC610F0FDC611F0FCC6E6FF9A
:100D8000FDC6E6FF290EE66EDC0EE926000EEA221D
:100D9000EECF12F0EFCF13F0010E1224E66E80ECCE
:100DA00009F0E552E552E552E552FCC6E9FFFDC601
:100DB000EAFFDC0EE926000EEA22EE6AED6A47D071
:100DC000FCC6E9FFFDC6EAFFE20EE926000EEA22B4
:100DD000EFCF10F0010E105C3AE3FCC6E9FFFDC650
:100DE000EAFFE20EE926000EEA22050EEFCFDBFF56
:100DF000FCC6E9FFFDC6EAFFE10EE926000EEA2285
:100E0000060EEFCFDBFFFCC6E9FFFDC6EAFFE00EF2
:100E1000E926000EEA22070EEFCFDBFFD950050FBF
:100E2000E66E000EDA20E66E280EE66E030EE66E23
:100E300080EC09F0E552E552E552E552FCC6E9FFC7
:100E4000FDC6EAFFE20EE926000EEA22EF6A090E6D
:100E5000E15C02E2E16AE552E16EE552E7CFD9FFDB
:100E60001200FCC6E9FFFDC6EAFFE80EE926000E07
:0C0E7000EA22EF50220801E1000C010C06
:040E7C00D9CFE6FFE5
:100E8000E1CFD9FFE652FD0EDBCFE9FFFE0EDBCF4F
:100E9000EAFF060EE926000EEA22EF6AFD0EDBCF1E
:100EA000E9FFFE0EDBCFEAFF070EE926000EEA227D
:100EB000EF6ADF6A030EDF5C15E2FD0EDBCFE9FFB0
:100EC000FE0EDBCFEAFFDF50020DE950F324E96E9E
:100ED000EA50F420EA6EEE50EFCFEAFFE96EEF6AD7
:100EE000DF2AE8D7E552E552E7CFD9FF1200050126
:100EF000FA6B000EEA6F0B0EEB6F000EEC6F0A0E32
:100F0000ED6F000EEE6F090EEF6F000EF26F080E20
:100F1000F36F000EF46F070EF56F000EF66F060EFE
:100F2000F76FEA0EE66E050EE66EA8DFE552E552B3
:100F3000F20EE66E050EE66EA1DFE552E5521200F6
:100F4000D9CFE6FFE1CFD9FF050EE126FC0EDB503D
:100F5000E66ED950030FE96EDACFEAFFE552E750AB
:100F6000EE6EED6AFD0EDBCFE9FFFE0EDBCFEAFF92
:100F7000060EE926000EEA22EFCFDFFFFD0EDBCFE3
:100F8000E9FFFE0EDBCFEAFFDF50020DE950F3244C
:100F9000E96EEA50F420EA6E010EEECFDBFF020E9E
:100FA000EDCFDBFF010EDBCFE9FF020EDBCFEAFF67
:100FB000EF5002E0FF0E64D0010EDBCFE9FF020E1E
:100FC000DBCFEAFFEE52FC0EDBCFEFFF010EDBCFF3
:100FD000E9FF020EDBCFEAFFE926000EEA22FB0E54
:100FE000DBCFEFFF030EDBCFE6FF040EDBCFE6FF28
:100FF000F90EDBCFE6FFFA0EDBCFE6FF010EDBCF0B
:10100000E9FF020EDBCFEAFF030EE926000EEA221B
:10101000E9CF10F0EACF11F0E9CFE6FFEACFE6FF23
:101020004BEC13F0126E060EE15E1250FD0EDBCF9C
:10103000E9FFFE0EDBCFEAFF060EE926000EEA22EC
:10104000EF28106E030E116E0C6E10C007F056ECF8
:1010500014F00350E66EFD0EDBCFE9FFFE0EDBCF92
:10106000EAFF060EE926000EEA22E552E750EF6E8F
:10107000010EDBCFE9FF020EDBCFEAFF010EEF6EC0
:10108000106E050EE15C02E2E16AE552E16E10507D
:10109000E552E7CFD9FF1200D9CFE6FFE1CFD9FF64
:1010A000050EE126FD0EDBCFE9FFFE0EDBCFEAFFEA
:1010B000070EE926000EEA22EFCFDFFFFD0EDBCFA1
:1010C000E9FFFE0EDBCFEAFFDF50020DE950F3240B
:1010D000E96EEA50F420EA6E010EEECFDBFF020E5D
:1010E000EDCFDBFF010EDBCFE9FF020EDBCFEAFF26
:1010F000EF0401E086D0010EDBCFE9FF020EDBCF6B
:10110000EAFFEE52EFCF10F0FC0EDB50D880105407
:1011100002E2FD0E77D0010EDBCFE9FF020EDBCF3E
:10112000EAFFEE52EF50E66ED950030FE96EDACFC8
:10113000EAFFE552E750EE6EED6A030EDBCFE6FF05
:10114000040EDBCFE6FF010EDBCFE9FF020EDBCFA3
:10115000EAFF030EE926000EEA22E9CF10F0EACFFB
:1011600011F0E9CFE6FFEACFE6FFF80EDBCFE6FFAE
:10117000F90EDBCFE6FF4BEC13F0126E060EE15ECC
:101180001250FD0EDBCFE9FFFE0EDBCFEAFF070EAC
:10119000E926000EEA22EF28106E030E116E0C6E87
:1011A00010C007F056EC14F00350E66EFD0EDBCFD6
:1011B000E9FFFE0EDBCFEAFF070EE926000EEA226A
:1011C000E552E750EF6E010EDBCFE9FF020EDBCFF9
:1011D000EAFFE926000EEA22EF50E66EFA0EDBCFB8
:1011E000E9FFFB0EDBCFEAFFE552E750EF6E010EA1
:1011F000DBCFE9FF020EDBCFEAFFEF6A030EDB5025
:1012000001D0FC0E106E050EE15C02E2E16AE552CF
:10121000E16E1050E552E7CFD9FF1200D9CFE6FFBB
:10122000E1CFD9FF030EE126FD0EDBCFE9FFFE0E75
:10123000DBCFEAFF070EE926000EEA22EFCFDFFF41
:10124000FD0EDBCFE9FFFE0EDBCFEAFFDF50020D24
:10125000E950F324E96EEA50F420EA6E010EEECF75
:10126000DBFF020EEDCFDBFF010EDBCFE9FF020E4D
:10127000DBCFEAFFEF040BE1010EDBCFE9FF020E4B
:10128000DBCFEAFFE926000EEA22EF5001D0000E84
:10129000106E030EE15C02E2E16AE552E16E10506D
:1012A000E552E7CFD9FF1200D9CFE6FFE1CFD9FF52
:1012B000FD0EDBCFE9FFFE0EDBCFEAFFE9CF10F03A
:1012C000EACF11F0FD0EDBCFE9FFFE0EDBCFEAFF28
:1012D000070EE926000EEA22EF50020D1050F3240B
:1012E000E96E1150F420EA6EEE50EFCFEAFFE96E9E
:1012F000EF50E552E7CFD9FF1200D38E0300120062
:10130000D9CFE6FFE1CFD9FFFB0EDBCFE6FFFC0E26
:10131000DBCFE6FFFD0EDBCFE6FFFE0EDBCFE6FF09
:10132000EA0EE66E050EE66E0BDE106E060EE15E50
:101330001050E552E7CFD9FF1200D9CFE6FFE1CF39
:10134000D9FFFA0EDBCFE6FFFB0EDBCFE6FFFC0E8C
:10135000DBCFE6FFFD0EDBCFE6FFFE0EDBCFE6FFC9
:10136000EA0EE66E050EE66E97DE106E070EE15E83
:101370001050E552E7CFD9FF1200EA0EE66E050ED7
:10138000E66E4CDFE552E5521200D9CFE6FFE1CF21
:10139000D9FFFB0EDBCFE6FFFC0EDBCFE6FFFD0E39
:1013A000DBCFE6FFFE0EDBCFE6FFF20EE66E050EAC
:1013B000E66EC6DD106E060EE15E1050E552E7CF18
:1013C000D9FF1200D9CFE6FFE1CFD9FFFA0EDBCF6C
:1013D000E6FFFB0EDBCFE6FFFC0EDBCFE6FFFD0EEC
:1013E000DBCFE6FFFE0EDBCFE6FFF20EE66E050E6C
:1013F000E66E52DE106E070EE15E1050E552E7CF4A
:10140000D9FF1200F20EE66E050EE66E07DFE5521A
:10141000E55212000501FA5101E11200EDEC0EF067
:10142000F3CF10F0F4CF11F0F350F41001E01200FC
:10143000D1EC0EF0F3CF10F0F4CF11F0F350F41024
:1014400001E11200EA0EE66E050EE66E2DDFE552B2
:10145000E552000901E012007DEF09F0F9EC0EF011
:10146000F3CF10F0F4CF11F0F350F41001E11200BB
:101470000501010EFA6FEA0EE66E050EE66E14DF48
:10148000E552E552000903E00501FA6B12000A0E6D
:0A149000E66E18EC14F0E552EED7FA
:06149A00D9CFE6FFE1CF0F
:1014A000D9FF9388939A8A988A9AFD0EDBCFFBF531
:1014B000FE0EDBCFFCF5FBC5E9FFFCC5EAFFF30E32
:1014C000E926000EEA22EF6AFBC5E9FFFCC5EAFF48
:1014D000F40EE926000EEA22EF6AFBC5E9FFFCC51F
:1014E000EAFFF50EE926000EEA220A0EEF6EFBC5B2
:1014F000E9FFFCC5EAFF030EE926000EEA22E9CF68
:10150000FDF5EACFFEF5E552E7CFD9FF1200D9CFBE
:10151000E6FFE1CFD9FFFE0EDB507E0823E1FBC5DD
:10152000E9FFFCC5EAFFF30EE926000EEA22EF6AA6
:10153000FBC5E9FFFCC5EAFFF40EE926000EEA222E
:10154000EF6AFBC5E9FFFCC5EAFF7E0EEF6EFBC547
:10155000E9FFFCC5EAFFF50EE926000EEA220B0EB4
:10156000EF6EB8D0FBC5E9FFFCC5EAFFF50EE92632
:10157000000EEA22EF500F0A01E192D0010A2EE09C
:10158000020A1AE0070A02E0010AA4D0FBC5E9FF3B
:10159000FCC5EAFFEE52010EE926000EEA22FE0E1D
:1015A000DBCFEFFFFBC5E9FFFCC5EAFFF50EE9263F
:1015B000000EEA220C0E8DD0FBC5E9FFFCC5EAFF48
:1015C000EE52FE0EDBCFEFFFFBC5E9FFFCC5EAFFE5
:1015D000F50EE926000EEA220E0E7BD0FBC5E9FFD0
:1015E000FCC5EAFFF30EE926000EEA22EFCF10F069
:1015F000FBC5E9FFFCC5EAFFEE52EECF11F0EFCFDD
:1016000012F01150105C000E125426E2FBC5E9FFE7
:10161000FCC5EAFFF30EE926000EEA22EF500501B1
:10162000EA6AFD25E96EFE51EA22FE0EDBCFEFFFEE
:10163000FBC5E9FFFCC5EAFFF40EE926000EEA222D
:10164000FE0EDB50EF26FBC5E9FFFCC5EAFFF30EFB
:10165000E926000EEA22EF2AFBC5E9FFFCC5EAFFF6
:10166000F30EE926000EEA22EF50106E116AFBC558
:10167000E9FFFCC5EAFFEE52EECF12F0EFCF13F018
:101680001250101827E11350111824E1FBC5E9FF8F
:10169000FCC5EAFFF50EE926000EEA220F0E19D06E
:1016A000FBC5E9FFFCC5EAFFF40EE926000EEA22BD
:1016B000EF28E86C106EFE0EDB50105C01E10ED8D6
:1016C000FBC5E9FFFCC5EAFFF50EE926000EEA229C
:1016D0000A0EEF6EE552E7CFD9FF1200D9CFE6FF31
:1016E000E1CFD9FFE652FDC5E9FFFEC5EAFFEF50A5
:1016F0008A0A40E01F0A38E0340A30E0360A28E05F
:10170000060A20E0030A18E0190A10E01B0A08E0A4
:10171000180A47E1FDC5E6FFFEC5E6FF3C0E2FD0E7
:10172000FDC5E6FFFEC5E6FF3D0E29D0FDC5E6FF7F
:10173000FEC5E6FF3E0E23D0FDC5E6FFFEC5E6FF73
:101740003F0E1DD0FDC5E6FFFEC5E6FF400E17D0DB
:10175000FDC5E6FFFEC5E6FF410E11D0FDC5E6FF63
:10176000FEC5E6FF420E0BD0FDC5E6FFFEC5E6FF57
:10177000430E05D0FDC5E6FFFEC5E6FF440EE66E4E
:10178000FBC5E9FFFCC5EAFFEE52EF50E66E80ECC8
:1017900009F0E552E552E552E552DF6EDFCF10F079
:1017A0001034E552E552E7CFD9FF1200D9CFE6FF5A
:1017B000E1CFD9FF020EE126010EDB6A7E0EE66E56
:1017C00001EC14F0E552A850020BFDE06BD80009C3
:1017D000FAE1E66A01EC14F0E552A850020BFDE0D4
:1017E00061D80009FAE1FC0EDBCFE6FF01EC14F052
:1017F000E552A850020BFDE055D80009FAE1DF6A76
:10180000FC0EDB50DF5C2DE2DF50E76EFD0EDBCF20
:10181000E9FFFE0EDBCFEAFFE750E926000EEA22E1
:10182000EF50E66E01EC14F0E552DF50E76EFD0E6E
:10183000DBCFE9FFFE0EDBCFEAFFE750E926000E23
:10184000EA22010EDBCFE7FFEF50E726010EE7CFDC
:10185000DBFFA850020BFDE025D80009FAE1DF2AE2
:10186000CFD7010EDB28E86CE66E01EC14F0E552F0
:10187000A8A2FED7020EE15C02E2E16AE552E16E47
:10188000E552E7CFD9FF1200D9CFE6FFE1CFD9FF6C
:10189000FE0EDB5002E08A8A01D08A9AE552E7CF39
:1018A000D9FF1200D9CFE6FFE1CFD9FFE652815030
:1018B000100B01E0010EDF6EDF5002E0010E01D0DF
:0C18C000000EE552E552E7CFD9FF120000
:0418CC00D9CFE6FF8B
:1018D000E1CFD9FF180EE126020EDB6A030EDB6AA8
:1018E000FC0ED3140009D36EF70EE66E040EE66EFE
:1018F000D0EC11F0E552E552000EE66E040EE66EF5
:101900004DEC0AF0E552E552000EE66E050EE66E6D
:101910001CEC00F0E552E55277EC07F0BEEC0DF060
:101920000DEC12F028EC14F080EC0FF0CDEC0EF082
:10193000C8EC0EF05F0EE66E71EC01F0E5522EEC95
:101940000AF0000EE66E0C0EE66ED950010FE66E40
:10195000000EDA20E66EDC0EE66E9DEC09F0106EED
:10196000050EE15E1050DF6EDFCF10F0103403E3A0
:10197000FC0EDF5CE4D7010EDB504D0AE0E0010A0B
:10198000DEE0070ADCE0010ADAE0030AD8E0010A37
:10199000D6E00F0AD4E0010AD2E0020A01E1D6D073
:1019A000070A01E1D0D0010A01E1CAD0030A01E12E
:1019B000C4D0010A01E1BED07F0A01E1B8D0010A1A
:1019C00001E1B2D0030A01E17BD0010A61E0120A11
:1019D000B6E0030A4FE0010AB2E0070AB0E0020AEB
:1019E00012E0010A03E0360AAAE0BAD0020EDB6A6E
:1019F000DF50F36E020EDBCFF4FFF350F45C9FE296
:101A0000020EDB2AF5D7020EDB6ADF04F36E020E4C
:101A1000DBCFF4FFF350F45C03E2020EDB2AF5D7D0
:101A20000C010051090A01E18AD7010A01E187D7B7
:101A30000F0A01E184D7010A01E181D7020A07E018
:101A4000060A01E07CD7010EDF6E006F05D0010EA3
:101A5000DF6E030EDBCF00FC000EE66E0C0EE66EB2
:101A60002A0EE66EDFCFE6FFC5EC09F0E552E5523F
:101A7000E55258D0020EDB6ADF50F36E020EDBCF68
:101A8000F4FFF350F45C01E35AD7020EDB2AF4D7DB
:101A9000D950040FE96EDACFEAFF000EEE6E0C0E9D
:101AA000ED6E020EDB6A050EDF5CF36E020EDBCF1D
:101AB000F4FFF350F45C01E342D7020EDB2AF3D7C4
:101AC000D950060FE96EDACFEAFF000EEE6E0C0E6B
:101AD000ED6E020EDB6A0C0EDF5CF36E020EDBCFE6
:101AE000F4FFF350F45C03E2020EDB2AF4D7060E97
:101AF000DBCFE9FF070EDBCFEAFF0C0EE926000E75
:101B0000EA22030EEFCFDBFF060EDBCFE9FF070E65
:101B1000DBCFEAFF0C0EE926000EEA22EF50E66E5C
:101B200027EC0EF0E5520BD7D950080F11D0D95041
:101B30000A0F0ED0D9500C0F0BD0D9500E0F08D071
:101B4000D950100F05D0D950120F02D0D950140F10
:101B5000E96EDACFEAFF000EEE6E0C0EED6EEFD6F8
:101B6000020EDB6ADF50F36E020EDBCFF4FFF350A0
:0C1B7000F45C01E3E4D6020EDB2AF4D79B
:041B7C00929092921F
:101B8000929492968990899289948996E66AE66AF7
:101B900008D8E552E55212008982000089920000BF
:101BA0001200D9CFE6FFE1CFD9FF020EE1268990DE
:101BB000DE6ADD6ADECF10F0DDCF11F0D890115073
:101BC00004E6080E105C000E115814E2FD0EDB5006
:101BD000010BE8B08984E8A08994DEDFFD0EDBCF3D
:101BE000F3FFF390F342F3CFDBFFDF2A010EE2E3D2
:101BF000DB2AE0D7DE6ADD6ADECF10F0DDCF11F040
:101C0000D890115004E6080E105C000E115814E232
:101C1000FE0EDB50010BE8B08984E8A08994BCDF9C
:101C2000FE0EDBCFF3FFF390F342F3CFDBFFDF2AAF
:101C3000010EE2E3DB2AE0D78980020EE15C02E2DA
:101C4000E16AE552E16EE552E7CFD9FF1200D9CF44
:101C5000E6FFE1CFD9FF030EE126DF6A010EDB6A62
:101C6000020EDB6A0A0E106E0C6EFE0EDBCF07F062
:101C700056EC14F0020E03C0DBFFDB50090A36E01D
:101C8000010A30E00F0A2AE0010A24E0030A1EE0FC
:101C9000010A18E0070A12E0010A0CE0030A06E054
:101CA000010A27E1010EE6C7DBFF23D0010EE7C7DB
:101CB000DBFF1FD0010EE8C7DBFF1BD0010EE9C719
:101CC000DBFF17D0010EEAC7DBFF13D0010EEBC715
:101CD000DBFF0FD0010EECC7DBFF0BD0010EEDC711
:101CE000DBFF07D0010EEEC7DBFF03D0010EEFC70D
:101CF000DBFF0A0E106E0C6EFE0EDBCF07F056EC0B
:101D000014F0020E07C0DBFFDB50090A2DE0010AC8
:101D100028E00F0A23E0010A1EE0030A19E0010A85
:101D200014E0070A0FE0010A0AE0030A05E0010ACD
:101D30001DE1E6C7DFFF1AD0E7C7DFFF17D0E8C70E
:101D4000DFFF14D0E9C7DFFF11D0EAC7DFFF0ED0F5
:101D5000EBC7DFFF0BD0ECC7DFFF08D0EDC7DFFF1D
:101D600005D0EEC7DFFF02D0EFC7DFFF010EDBCFEC
:101D7000E6FFDFCFE6FF15DFE552E552030EE15C3B
:101D800002E2E16AE552E16EE552E7CFD9FF1200C7
:101D9000A58A9F86F08C9D861200D08EF28EF29CD2
:101DA0001200F250800B800A01E0010E106E116AE1
:101DB00010BE116810C0F3FF11C0F4FF1200F25002
:101DC000400B400A01E0010E106E116A10BE11684E
:101DD00010C0F3FF11C0F4FF1200F2BC04D0E1DF29
:101DE000F350F41002E0F36A02D0010EF36EF46ACD
:101DF0001200F3DFF3CF10F0F4CF11F0F350F41032
:101E000007E1CFDFF350F41003E1010EF36E01D0D0
:101E1000F36AF46A1200DACFE4FFE2CFDAFFE9CF27
:101E2000E4FFEACFE4FFF6CFE4FFF7CFE4FFF8CF1B
:101E3000E4FFF5CFE4FFF3CFE4FFF4CFE4FFFACF04
:101E4000E4FFFBCFE4FF00EE00F0100EE80403E334
:101E5000EECFE4FFFBD700EE10F0050EE80403E33D
:101E6000EECFE4FFFBD7E6529EA60CD0010EE66E45
:101E700044EC0CF0E5529E9693EC01F0E66A44ECDB
:101E80000CF0E552A4AA03D0F1EC11F0A49AE552AB
:101E900000EE14F0050EE80403E3E5CFEDFFFBD7F9
:101EA00000EE0FF0100EE80403E3E5CFEDFFFBD7E3
:101EB000E5CFFBFFE5CFFAFFE5CFF4FFE5CFF3FF7A
:101EC000E5CFF5FFE5CFF8FFE5CFF7FFE5CFF6FF6C
:101ED000E5CFEAFFE5CFE9FFE5CFDAFF1100D8CF84
:101EE000E4FFE0CFE4FFE46EDACFE4FFE652E55230
:101EF000E5CFDAFFE550E5CFE0FFE5CFD8FF1000F2
:101F0000928A94948B940E01100EE16FF086F19AF0
:101F100012008B84640EE66EEAEC13F0E5528B94AB
:101F2000120004010F0EF96FF19E9388938A938C2F
:101F3000938E8A988A9A8A9C8A9EF2861200D9CFBA
:101F4000E6FFE1CFD9FFE652F00E8114E8380F0B1F
:101F5000DF6EDF500401F919010B13E0F9A105D080
:101F6000000EE66EE66A470E04D0000EE66EE66AE4
:101F7000460EE66EE66A80EC09F0E552E552E5525F
:101F8000E552DF500401F919020B13E0F9A305D063
:101F9000000EE66EE66A490E04D0000EE66EE66AB2
:101FA000480EE66EE66A80EC09F0E552E552E5522D
:101FB000E552DF500401F919040B13E0F9A505D02F
:101FC000000EE66EE66A4B0E04D0000EE66EE66A80
:101FD0004A0EE66EE66A80EC09F0E552E552E552FB
:101FE000E552DF500401F919080B13E0F9A705D0F9
:101FF000000EE66EE66A4D0E04D0000EE66EE66A4E
:102000004C0EE66EE66A80EC09F0E552E552E552C8
:10201000E552DFCFF9F4E552E552E7CFD9FF1200E0
:10202000D9CFE6FFDACFE6FFE1CFD9FFE2CFDAFF83
:10203000E652E652E652DF6AF8CF01F0F6CF02F040
:10204000FD0EDB80DB82DB84DB86DB88DB8AFC0E3B
:10205000DB84DB86DB88DB8ADB8CDB8EFD0EDBCF73
:10206000E6FFC00EBA10E552E714BA6EFC0EDBCFE5
:10207000E6FF0F0EBA10E552E714BA6E3F0E106E6F
:10208000FD0EDB50105C02E194940FD0FD0EDB508E
:10209000BF0802E1949409D0FD0EDB507F0804E0F4
:1020A000FD0EDB50FF0801E1949401C0F8FF02C06F
:1020B000F6FFE552E552E552E552E5CFDAFFE7CF0C
:0420C000D9FF120032
:0C20C400D9CFE6FFDACFE6FFE1CFD9FF6D
:1020D000E2CFDAFFC26AC16AFC0EDB50400DF3505A
:1020E000C00B106EFC0EDB407F0B3C0B1010C26E61
:1020F000FD0EDB50040DF350380B116EFD0EDB3876
:102100000F0B070B106EFD0EDB50800B1010111023
:10211000C16EF90EDBCF10F0FA0EDBCF11F011C05B
:1021200010F0116A10C048FFF90EDBCF49FF060E10
:10213000106EFB0EDB50C00B10C0E7FFE75204E04F
:10214000E8427F0BE706FCE10E01B86FFC0EDBAE48
:1021500003D09E9C9D8CF28CC280E552E5CFDAFFC5
:06216000E7CFD9FF1200D9
:0A2166001E0EF66E000EF76E000E5E
:10217000F86E06010900F550F56F0900F550F66F8D
:1021800003E1F56701D03DD00900F550F06F09007B
:10219000F550F16F0900F550F26F09000900F55094
:1021A000E96E0900F550EA6E090009000900F550D2
:1021B000F36F0900F550F46F09000900F6CFF7F648
:1021C000F7CFF8F6F8CFF9F6F0C6F6FFF1C6F7FF4D
:1021D000F2C6F8FF0601F35302E1F45307E00900E9
:1021E000F550EE6EF307F8E2F407F9D7F7C6F6FFFD
:1021F000F8C6F7FFF9C6F8FF0601F507000EF65B13
:04220000BFD7120032
:0C220400D9CFE6FFDACFE6FFE1CFD9FF2B
:10221000E2CFDAFFE652E652E652DF6AF8CF01F08B
:10222000F6CF02F0FD0EDB80DB82DB84DB86DB8811
:10223000DB8AFC0EDB84DB86DB88DB8ADB8CDB8ED7
:10224000FD0EDBCFE6FFC00EB410E552E714B46E0E
:10225000FC0EDBCFE6FF0F0EB410E552E714B46EB0
:102260003F0E106EFD0EDB50105C01E10DD0FD0E37
:10227000DB50BF0801E108D0FD0EDB507F0804E011
:10228000FD0EDB50FF0800E101C0F8FF02C0F6FFC1
:10229000E552E552E552E552E5CFDAFFE7CFD9FF47
:0222A00012002A
:0E22A200D9CFE6FFDACFE6FFE1CFD9FFE2CFDA
:1022B000DAFF0C0EBA6EFC0E0F015217DB50180B32
:1022C000E840E840E8401F0B5213070E521506E1A4
:1022D000CA94FD0EDB50CB6ECA841DD0070E52157A
:1022E000010806E17694FD0EDB50776E768413D0FC
:1022F000070E5215020806E11E95FD0EDBCF1FFFEB
:102300001E8509D0070E5215030805E11B95FD0E29
:10231000DBCF1CFF1B85E552E5CFDAFFE7CFD9FF06
:022320001200A9
:0E232200D9CFE6FFDACFE6FFE1CFD9FFE2CF59
:10233000DAFF0C0EB46EC70E0F015217FC0EDB5005
:10234000700BE8407F0B5213380E521506E1CA9409
:10235000FD0EDB50CB6ECA841DD0380E5215080816
:1023600006E17694FD0EDB50776E768413D0380E3E
:102370005215100806E11E95FD0EDBCF1FFF1E85CE
:1023800009D0380E5215180805E11B95FD0EDBCF5C
:102390001CFF1B85E552E5CFDAFFE7CFD9FF12001E
:1023A000D9CFE6FFE1CFD9FF190EE66EE66A3C0E03
:1023B000E66E86EC12F0E552E552E5520E010A0E89
:1023C000F76F060EC96F190EE66EE66A7C0EE66EB2
:1023D0004AEC12F0E552E552E552E552E7CFD9FF5B
:1023E0001200A4AA06D076EC13F0E66E87EC0AF091
:1023F000E5520501FFA710D0AC98AC889C989C884A
:10240000000EE66EE66A1E0EE66EE66A80EC09F0E5
:0A241000E552E552E552E5521200D4
:06241A00949094928B9057
:102420008B920E010E0ECB6F120ECC6F12008F0E20
:10243000E66EE66851EC11F0E552E552F40EE66EF8
:10244000010EE66EEEEC12F0E552E552FC0EE66E81
:102450003F0EE66E10EC10F0E552E5528F0EE66E80
:10246000E66891EC11F0E552E552F40EE66E010ECD
:10247000E66EBFEC12F0E552E552FC0EE66E3F0E42
:10248000E66E02EC11F0E552E55212006DEC14F02C
:042490000AEF00F05F
:0C249400D9CFE6FFDACFE6FFE1CFD9FF99
:1024A000E2CFDAFFA86A9C6AFD0EDBB0A888DBA247
:1024B00002D0A88C9C8CDBB4A88EDBA602D09C88B2
:1024C00001D09C8ADBA802D0A88401D0A894DBBAF2
:1024D0009C86DBAC02D0A38A01D0A39ADBAE02D0EB
:1024E000A38801D0A398FB0EDB50AB6EFC0EDBCFB4
:1024F00011F011C010F0116A10507D6EA88A9C8EE8
:0C250000E552E5CFDAFFE7CFD9FF12006B
:04250C00D9CFE6FF3E
:10251000DACFE6FFE1CFD9FFE2CFDAFFAD6AAC6AEE
:10252000FD0EDBB0AD88DBA202D0AD8CAC8CDBB491
:10253000AD8EDBA602D0AC8801D0AC8ADBB8AD840E
:10254000DBBAAC86DBAC02D09D8A01D09D9ADBAEB3
:1025500002D09D8801D09D98FB0EDB50B06EFC0E22
:10256000DBCF11F011C010F0116A10507F6EAD8AF0
:0E257000AC8EE552E5CFDAFFE7CFD9FF1200BF
:02257E00D9CFB3
:10258000E6FFDACFE6FFE1CFD9FFE2CFDAFFE6528E
:10259000E652FC0EDBCF10F0FD0EDBCF11F0060E85
:1025A000D89010361136E804FBE110C0DEFF11C0F0
:1025B000DDFF010EDB50B56EDF50E840E8403F0B19
:1025C000300B106ECF0EB4141010B46EE552E552FD
:0C25D000E552E5CFDAFFE7CFD9FF12009B
:0425DC00D9CFE6FF6E
:1025E000DACFE6FFE1CFD9FFE2CFDAFFE652E652DB
:1025F000FC0EDBCF10F0FD0EDBCF11F0060ED890F5
:1026000010361136E804FBE110C0DEFF11C0DDFF1B
:10261000010EDB50BB6EDF50E840E8403F0B300B53
:10262000106ECF0EBA141010BA6EE552E552E55294
:0A263000E5CFDAFFE7CFD9FF120073
:06263A009280FE0EE66E28
:102640001F0EE66EE66A840EE66EE10EE66E62EC42
:1026500010F0106E050EE15E105012006FEF14F0D6
:1026600007EF00F0D9CFE6FFE1CFD9FF030EE12657
:1026700064EC14F0F3CFDEFFF4CFDDFF020EF36E57
:10268000DB6E030EE15C02E2E16AE552E16EE552C7
:06269000E7CFD9FF1200A4
:0A269600D9CFE6FFDACFE6FFFA0E17
:1026A000E3CFD9FFFB0EE3CFDAFFFC0EE3CFE9FF68
:1026B000FD0EE3CFEAFFE9CFF3FFEACFF4FFF80E18
:1026C000E35003E1F90EE35008E0F80EE30602E2FE
:1026D000F90EE306DECFEEFFF2D7FF0EE3CFDAFF0F
:0C26E000E552FF0EE3CFD9FFE5521200D7
:0426EC00D9CFE6FF5D
:1026F000DACFE6FFE1CFD9FFE2CFDAFFE652F20E02
:102700000501FF179CAC03D0FF919CB0FF819CB4E6
:10271000FF859CB2FF87AA50DF6EDF50E552E5527D
:0A272000E5CFDAFFE7CFD9FF120082
:06272A00FEC6E9FFFFC638
:10273000EAFFEF6AFEC6E9FFFFC6EAFFEE52EF6A64
:10274000FEC6E9FFFFC6EAFF020EE926000EEA22F6
:10275000EF6AFEC6E9FFFFC6EAFF030EE926000E98
:06276000EA22EF6A1200FC
:0A276600D9CFE6FFDACFE6FFE1CF9E
:10277000D9FFE2CFDAFFE652E652FC0EDBCFDEFFF6
:10278000DBCFDDFF010EDB50CF6EDF50CE6EE552AA
:0E279000E552E552E5CFDAFFE7CFD9FF1200A0
:02279E00D9CF91
:1027A000E6FFDACFE6FFE1CFD9FFE2CFDAFFFD0E99
:1027B000DB50FB0BCA6ECC6A9E92FD0EDBAE02D0E4
:1027C0009D8201D09D92CA84E552E5CFDAFFE7CF22
:0427D000D9FF12001B
:0C27D400FF0EE350166EEF0E01D0F30E66
:1027E000E76EE72EF1EF13F00C0E156EE76AE72E99
:1027F000F7EF13F0152EF6EF13F0162EEFEF13F0A0
:022800001200C4
:0E280200D9CFE6FFDACFE6FFE1CFD9FFE2CF74
:10281000DAFFA8AC04D0A8900501FFB3A880FD0E94
:10282000DB50A96EE552E5CFDAFFE7CFD9FF120002
:10283000FF0EE350166E480E01D04C0EE76EE72EE9
:10284000FED7E76AE72EFED7162EF7D70000120054
:10285000050EE66ECFEC13F0E55212001200330EB7
:10286000E66EF30EE66EB3EC13F0E552E55212009D
:10287000B00EF36E00EE00F00E0E01D81200EA600A
:1028800002D0EE6AFCD7F350E9601200EE6AFCD782
:102890001DEE00F02DEE00F0F86A0F9CB3EC10F086
:0C28A00003EC00F066EC0CF0FBD712001B
:0428AC00036A080EA5
:1028B000E76ED890073603360C50035C02E3036ED4
:0828C000072AE72EF7D71200EA
:0828C800C450136E126AC350E4
:0A28D0001210F36E13C0F4FF1200A3
:0428DA00BA6A1200C4
:0228DE00C282B4
:0228E0001200E4
:0E28E20000EEFE9CFC9E8EFC60DAF266B6BE36
:0328F000E4FEF60D
:0D28F30000EEFE9CFC9E8EFC60DAF266B6E4
:04290000BEE4FEF63D
:020000040001F9
:01FFF800AA5E
:01FFFA00FD09
:01FFFD00F80B
:00000001FF
